:1000000002015C02018200000000003200000000DA
:10001000000000320000000000000032000000007C
:100020000000003200000000000000000000C39546
:10003000F02212002E60044002E422740122020029
:1000400041C3EDB50706ECB50602E4227401227B3C
:100050000474FA11FADBFADAF622C0E0740311FA3A
:10006000D0E0220022D2B51163D2B011637F0AD34F
:1000700030B50C30B009DFF8C2B01163C2B5C3921D
:100080000422C2B01163D2B51163D2B02292B01172
:1000900063500C7F0A20B007DFFBD2B5D38013D2A8
:1000A000B511637F0A20B507DFFBD2B0D38003C24E
:1000B000B5C322D2B01163D2B511637F0A20B50552
:1000C000DFFBD38007A2B092D5C2B5C3227E08332E
:1000D000118D400CDEF911B34006A2D550021182F9
:1000E00092042233FD7E0811B3400CA2D533DEF713
:1000F000CD13CD118DD2B092042278A37901D8FE10
:10010000D9FCD5E0F522EC2EFCED3FFD22312BECA5
:100110008EF0A4F8A9F0EC8FF0A429F9ED8EF0A4EC
:1001200029FDAC0030D50312015022C2D5C004C055
:1001300005AC06AD07ED30E709B2D5120150AE04AB
:10014000AF05D005D004ED30E705B2D5120150223D
:10015000EDF4FDECF42401FC50010D22787FE4F66F
:10016000D8FD7581407520007590FF75B0FFC2B451
:10017000D2AFD2A8C294C295C296C2974387020258
:100180000174D294D295D296D297753000752F0013
:10019000753200752300752400752B000532D2944A
:1001A000C29775220C300505309312C20520930DBD
:1001B00074281200FA209305D20512031C75220A36
:1001C000300605309212C20620920D74281200FAF1
:1001D000209205D20612031C75220B3007053091C0
:1001E00012C20720910D74281200FA209105D2073F
:1001F00012031CD297C2967522093005053093125E
:10020000C20520930D74281200FA209305D205121E
:10021000031C752208300605309212C20620920D8A
:1002200074281200FA209205D20612031C752207C8
:10023000300705309112C20720910D74281200FA80
:10024000209105D20712031CD296C2957522063062
:100250000505309312C20520930D74281200FA2070
:100260009305D20512031C75220530060530921243
:10027000C20620920D74281200FA209205D20612AE
:10028000031C752204300705309112C20720910D1E
:1002900074281200FA209105D20712031CD295C2CD
:1002A00094752203300505309312C20520930D7416
:1002B000281200FA209305D20512031C7522023081
:1002C0000605309212C20620920D74281200FA2000
:1002D0009205D20612031C752201300705309112D7
:1002E000C20720910D74281200FA209105D207123E
:1002F000031C300805209012C20830900D7428129B
:1003000000FA309005D2081204CA740A11FAE532D4
:10031000B4FA028002500302019C3222753200D2EC
:10032000B3746411FAC2B3743211FAA293920450F6
:1003300003020339740102033AE4C0E0A29292047A
:10034000500302034A740102034BE4D0F045F0C0AD
:10035000E0A2919204500302035F7401020360E47F
:10036000D0F045F0B40102800302036F02032BE5D5
:100370002FB40102800302037C0203D5E52FB402EF
:10038000028003020389020404E522B40B02800305
:10039000020399052F752B0022E522B40C0280037D
:1003A0000203D2B16BAC23AD247E0A7F00113E6004
:1003B000030203BA0204530203D2AC23AD24AE25D8
:1003C000AF26113E60030203CF0204A20203D20251
:1003D0000453020419E522B40C028003020401B1A3
:1003E0006BAC23AD24AE25AF26113E70030203F3A0
:1003F0000204539174752300752400752B00052F9A
:1004000022020419E522B40C02800302041975309B
:100410000191F891747532FC22052BE52BB404028E
:100420008002500302042A020453AC23AD247E0A46
:100430007F00310D8C238D24AC23AD24AE227F00B0
:1004400031068C238D24C0E0782BE62435F8D0E0EB
:10045000A622220531752D09752E5F917DE531B4F7
:10046000030280030204707A3C114F7531009174CD
:100470007532FC22752D02752EC8917D22752C01D6
:10048000852DF0E52C113270030204A1C2B3E52ED4
:1004900011FAD2B3E52E11FA052CE52C6003020403
:1004A00080227531007523007524009174D2B47ACE
:1004B00002114FC2B47A01114F7532FC78331678AD
:1004C00036A633752B0175300D227A04114FA29098
:1004D000920450030204DA0204F478367601783785
:1004E00076027838760378397604752B04753001F6
:1004F00091F891747532FC228530F0740AA4C0E042
:100500007834D0E0F6752D01852BF0E52D11327091
:1005100003020548852DF0E53425F0C0E07835D09C
:10052000E0F6782DE62435F8E6F52E116574A01175
:10053000CDE53511CDE52E11CD1182740A11FA05E4
:100540002DE52D600302050875F009E53425F0C09E
:10055000E07835D0E0F6116574A011CDE53511CD08
:10056000E52B11CD1182740A11FA22752C01852C0C
:10057000F0740AA4C0E07834D0E0F6782CE62324A6
:1005800023F8E4F608F675F009E53425F0C0E078C4
:1005900035D0E0F6116574A011CDE53511CD1165AA
:1005A00074A111CDD311E3F5F085F02E1182852EC3
:1005B0002B752D01852BF0E52D1132700302062DD0
:1005C000852DF0E53425F0C0E07835D0E0F61165F2
:1005D00074A011CDE53511CD116574A111CDD311E4
:1005E000E3F5F085F02E1182782CE6232423F8869B
:1005F000040886057E0A7F00310D782CE62324232B
:10060000F8A60408A605782CE6232423F886040817
:100610008605AE2E7F003106782CE6232423F8A62B
:100620000408A605052DE52D60030205B4227535E5
:1006300083116574A011CDE53511CD116574A1113B
:10064000CDD311E3F5F085F02E1182852E332200F3
:00000001FF
